:030000000219FDE5
:03000B000200A848
:03002B0002015D72
:03005B000202DCC2
:030073000202C2C4
:1000800002030406080C10182030406080040608A3
:100090000C10182030406080A0C000070F1F3F05E3
:1000A000050D050205030302C2AFC0D0C0E0206207
:1000B00017E5256002E473E525F4F58A758B00D217
:1000C00062D0E0D0D0D2AF3285268AC262E526F473
:1000D000602F758B00D0E0D0D0D297D295D293D23A
:1000E000AF32D297D295D293206E0C206609740558
:1000F000D5E0FDE57E4290758B00D0E0D0D0D2AF48
:1001000032758A00C28DD26201F701B730680520CE
:100110006602C29701B7306805206602C29301B734
:10012000306805206602C29501B7C29630680A2081
:1001300066077428D5E0FDC29701B7C29230680AFD
:100140002066077428D5E0FDC29301B7C2943068D9
:100150000A2066077428D5E0FDC29501B7C2AFC278
:10016000AD53E6EFC0D0C0E0D2D3D2AFC2CEE52AC5
:100170006007207449152A21BE7800790020742E6A
:10018000E580307E01F430E50278FF53DACF207E3F
:100190000343DA20307E0343DA10C2D8C271E5800F
:1001A000307E01F430E50279FFC3E89970CB30610D
:1001B00003752A18207403752A18885FD27020747A
:1001C0000DE52B6004152B21CE43DA01C2D8207037
:1001D000024130A85F206102C270207431C3E894EC
:1001E000F0400374F0F8E8C4540F28F87984B7039A
:1001F00002410EC313C3138721200802C313200A30
:1002000006C3C898F8410E28F8500374FFF8C3E8F5
:1002100095685003E568F88822E52D54066011E5DD
:1002200033C313C31324062522F52250037522FF7E
:10023000852224A824C3E52495644002A864882567
:10024000E56970024174C3E8AA699A5003E8FAE4C8
:10025000F9EAC333FBE56BF45B29400D256AF8E549
:100260006A6002156A400B41740AC3E56A9A50023B
:10027000056A78FF8826C3E52594404002D26420B1
:10028000CF0AD0E0D0D043E610D2AD32C2CF053A8B
:100290007801E52A6005307402152AC3E55F9401F0
:1002A000400575620041B8756300756C00E5622415
:1002B00001F56250037562FFD0E0D0D043E610D262
:1002C000AD32C2AFC0D053E67FC260759100855693
:1002D00094855795759104D0D0D2AF32C2AF53E612
:1002E000EFC2ADC0D0C0E0C0F0D2D3D2AFA8FBA95E
:1002F000FCC2D8307102614353DACF207E0343DA67
:1003000010307E0343DA20D271E580307E01F42084
:10031000E502611A88278928A17053DACF207E036D
:1003200043DA20307E0343DA10C2D8C2713074023F
:10033000A15C7800E580307E01F430E502A15C88A4
:100340005FA14453DACF207E0343DA20307E03439B
:10035000DA10C271206102811C53DACF207E034380
:10036000DA10307E0343DA20C2D8D271885A895B12
:10037000C3E89558F8E99559F97B007E087A00C3DF
:10038000E8948CE994005005755E00810E88217810
:10039000A2E6A8216055C3E894C8E994005008E497
:1003A000D2E4FB7A0A61E9C3E89468E99401500851
:1003B000E4D2E3FB7A0F61E9C3E894D0E9940250F8
:1003C00008E4D2E2FB7A1E61E9C3E894A0E994054F
:1003D0005008E4D2E1FB7A3C61E9C3E89498E994DF
:1003E000085008E4D2E0FB7A787E00C3E8955CFC14
:1003F000E9955DFD30E70AECF42401FCEDF43400EE
:10040000FD755E00C3EC9AED9E5003755E01885C3D
:10041000895D855A58855B597802A144C3E89527C0
:10042000F8E99528F9307C02A128307B02A1283018
:100430007A02A121207502813FE9FDE8FC815EE995
:10044000C313F9E813F8307902A121E9C313F9E8DD
:1004500013F8307802A121E9C313FDE813FC2061F1
:100460002CC3EC941CED940240028175ED701EC308
:0E047000EC94C850180529E52970021529C31F
:10047E00E529940A5002A15C755F00D270A15CE57B
:10048E0029600215297888E6F97400207F0878968D
:10049E00B90302789EE624FAFEE43400FFC3EC9E14
:1004AE00FCED9FFD9208B90310A2085007207609B3
:1004BE00D27681C7307602C276A2085016B9030DE5
:1004CE00ECF42401FCEDF43400FD0204E178007933
:1004DE0000A128B90315EC33FCED33FDC3EC940AEF
:1004EE00FCED9400FD50047C007D00C3EC94FFED08
:1004FE009400400678FF7900A128EC8575F0A4C51C
:10050E00F0A2F733F87900400302054478FF790032
:10051E00020544E9C313F9E813F8307C0EE96002D2
:10052E0078FFC3E81338F8E43400F9C3E894FFE920
:10053E009400400278FF885FD270206102A15C7443
:10054E001FF4552F4BF52FC274EB7002D274752A1F
:10055E0018307403752A0A306102A1702074035397
:10056E00DAFE207403752B06D0F0D0E0D0D0D2ADD9
:10057E0043E6103279010205A079030205A0790A3B
:10058E000205A0791E0205A079640205A079C802B1
:10059E0005A07817E4D5E0FDD8FAD9F6227A147BB7
:1005AE00780205C77A107B8C0205C77A0D7BB402E0
:1005BE0005C77A0B7BC80205C77902B27DE4C292E9
:1005CE00D5E0FDC293D5E0FDD293D5E0FDD292D514
:1005DE00E0FDC297E576D5E0FDD2977496D5E0FDA5
:1005EE00D9D9EAF8D5E0FDD8FBDBCEC29222C37C86
:1005FE00007D0075F00005F0EA33FAEB33FB50F6A0
:10060E00EB13FBEA13FAC3E9FFE8FEE89AF8E99B5D
:10061E00F95004EFF9EEF8B3EC33FCED33FDD5F001
:10062E00DFEDF9ECF822E889F08A20D2D4F8A9F0AF
:10063E007B0030F70B7BFFF42401F8E9F43400F96A
:10064E00E88520F0A4ADF0F8E98520F0A4AFF0FE27
:10065E00ED2EF974003FFA7C04C3EA13FAE913F99C
:10066E00E813F8DCF48BF030F70AE8F42401F8E92B
:10067E00F43400F9E889F0C2D4F8A9F02222C3E5D7
:10068E004113F9E54013F8C3E54598F8E54699F9A5
:10069E00500CC3E89480E994FF40160206C3C3E8E9
:1006AE00947FE9940050030206C3787F7900020616
:1006BE00C3788079FF884A894B22E54A2547F8E5B9
:1006CE004B3548F9854B20E4300701F43549FA30B3
:1006DE00E709C3EA94F04015020701C3EA940F50EC
:1006EE000302070178FF79FF7A0F0207017800797C
:1006FE00007AF0C3E5249564500AC3740195245022
:10070E000B02071FE54B20E70E02071FE54B30E7F4
:10071E0006884789488A492278A4E6FAC3E54A330F
:10072E00F8E54B33F9D134E930E70BC3E89480E9AF
:10073E0094FF4013E159C3E8947FE994005002E11D
:10074E0059787F7900E159788079FFE820E715C361
:10075E00E52398F84009C3E8940140030207807826
:10076E0001020780E8F424012523F84003020780E4
:10077E0078FF884C2278A5E6FAA848A949D134E931
:10078E0030E70CC3E89401E994FF40160207B4C3A6
:10079E00E894FFE9940050030207B478FF79000251
:1007AE0007B4780179FFE920E715C3E54C98F840C6
:1007BE0009C3E8940140030207DB78010207DBE876
:1007CE00F42401254CF840030207DB78FF8824222D
:1007DE0078FFC26420693D206A12D264C3E5419459
:1007EE000A4009C3E52594405002C26479A1E7602E
:1007FE0023E541601F74FF8541F0848539F0306A2E
:10080E000375F005A4F8C5F0600278FFC3E895679C
:10081E005002A867886622C3E5409440E5419401E2
:10082E00E5665003140136046002F5662202083EA6
:10083E002275E890227883E6FFE5E820ECF7A8BD64
:10084E00A9BE0573C3E57394084052757300E9FAA7
:10085E0079A0E76044EA7007E574601B020879C36B
:0F086E00E895746010E5745006600C140208855C
:10087D000460F9020885E574F574C3946D401B7529
:10088D0064C0C394044013756480C39404400B7515
:10089D006440C39404400375640075BB0822E5648D
:1008AD00F460020564E573B4070375BB102274325E
:1008BD0079A687F0A4C5F0A2F733F8C3E895644094
:1008CD0002A8648822882488258826886722754096
:1008DD00007541F022C2AF75C820A8CCA9CDAA3AA7
:1008ED0030CF010A75C824D2AFAB3BAC3C883B89F5
:1008FD003CC3E89BF8E99C206908F930670221F7B1
:10090D002154AD3D8A3DF9EA9DFA600478FF79FFE7
:10091D00AE3EAF3F8B3E8C3FC3EC9FFCC3E99CF5D5
:10092D0042A83BA93CC3E89EF8E99FF9C3E54113F2
:10093D00FBE54013FAE82AF540E93BF54150067511
:10094D0040FF7541FF219EAA40AB41AC40AD417EB9
:10095D00047F02C3EB940440021E1FC3EB940840B6
:10096D00021E1FC3ED13FDEC13FCDEF7C3EA9CFA68
:10097D00EB9DFBEF6009C3E913F9E813F8DFF7EA24
:10098D0028FAEB39FB8A408B4150067BFF8B408B5D
:10099D0041C3EB94025002D2673069047F0321C931
:1009AD007892E6FFC3E537948240110FC3E5379483
:1009BD00A040010FC3EF940640027F057E07E5417D
:1009CD00C4540FF9E541C454F0F8E540C4540F2860
:1009DD00F8C3E89EFAE99400FB4009C3EA9402EBE0
:1009ED00940050047A02E4FB4143AA40AB41EBC4AE
:1009FD00FEEAC4540F4EFCC3EA9CFAEB9400FBC311
:100A0D00E813C313F8EA28FAEB3400FB8A408B4154
:100A1D00C3EB94024002C2677807EBC4FE7B00EA89
:100A2D00C4540F4EFAC3EA98FA4005C3940250021B
:100A3D007A027892E6FF3060024143855256855323
:100A4D0057D26043E680C3E49AF8E49BF93067021D
:100A5D0041DDE8FAE9FBD3E913FDE813FC8852897F
:100A6D0053C3EF94036038EF20E00DE82CF8E93D17
:100A7D00F9ECFAEDFB020A98E828F8E939F9C3E830
:100A8D002402F8E93400F97AFE7BFFC3EF940340AA
:100A9D000E8A548B55884E894F8C508D516111881B
:100AAD005489558A4E8B4F8C508D51306920C3E53A
:100ABD003394034019E542A2E713F8E555F42401F8
:100ACD0038400B20E7087554FFF42401F5556111EA
:100ADD00E8FAD3E813FC8852C3EF94036020EF20AB
:100AED00E007E82CF8ECFA41FDE8282402F87AFE3C
:100AFD00C3EF940340088A54884E8C50611188547A
:100B0D008A4E8C50E56BC3335002646BF56B3060CD
:100B1D0002611B753402D26043E680E52D540660F8
:100B2D0026A840A941C3E913F9E813F8C2AF53E66B
:100B3D007F759100C3E498F594E499F5957591044A
:100B4D00D26043E680D2AF22D26575440075200095
:100B5D00306B03752040020B74D26575440075200F
:100B6D0040306B03752000D2AF7801206722E52D50
:100B7D0054066002C265C3E54194054013780294A2
:100B8D000540087803940540027806306902780A1A
:100B9D00206019E544601530690AC3E533940340BC
:100BAD0003D53406D2AFD26C81457123D2AF00008C
:100BBD00C2AF206726E541C3FB940F40027B0FEBCC
:100BCD00240530730123306A02742820620123F951
:100BDD003069027982E58BC39940B50544E59B5494
:100BED0040B52002812F30690A08C3E8940A4001FC
:100BFD0008619D2065026174C26553E67F759100A1
:100C0D003067107594007595FE759104D26043E6BA
:100C1D00806174AE40AF41C3E49EF594E49FF595B9
:100C2D008116C3E53394025002617430650261741C
:100C3D00D8028143619DC26C53E67F759100855446
:100C4D0094855595759104854E56854F57D26043C1
:100C5D00E680D2AFE52D54066008206A0205330206
:0F0C6D000C7F306C0D206B0A20650715811581F7
:100C7C000214F62278003064053065027801E537FD
:100C8C0075F007A4F9E5F028F5F0E9A2F013A2F14C
:100C9C0013A2F213F537C394785003753778C3E574
:100CAC003795384008D266D297D295D293306002ED
:100CBC0081B9855056855157D26043E68022207DFC
:100CCC0011C2AF754302C292D296D2AF759F130276
:100CDC000E99C2AF754302C292D294D2AF759F13D4
:100CEC00020E99307243207D20C2AF7543039001F0
:100CFC003B757E04D295C294306204C293A10DD28E
:100D0C0092D2AF759F10020E99C2AF75430390013A
:100D1C003B757E04D297C296306204C293A12DD249
:100D2C0092D2AF759F11020E99207D17C2AF7543F9
:100D3C0003900116D295306202C293D2AF759F1008
:100D4C00020E99C2AF754303900116D2973062021E
:100D5C00C293D2AF759F11020E99207D11C2AF754F
:100D6C004304C296D294D2AF759F11020E99C2AFB2
:100D7C00754304C294D296D2AF759F10020E99306F
:100D8C007243207D20C2AF75430590012A757E40C9
:100D9C00D293C292306204C297A1A9D296D2AF75F7
:100DAC009F13020E99C2AF75430590014C757E10CE
:100DBC00D293C292306204C295A1C9D294D2AF75BB
:100DCC009F13020E99207D17C2AF75430590010C3D
:100DDC00D293306202C297D2AF759F13020E99C2A2
:100DEC00AF754305900120D2933062EBC295D2AF20
:100DFC00759F13020E99207D11C2AF754306C294E4
:100E0C00D292D2AF759F10020E99C2AF754306C233
:100E1C0096D292D2AF759F11020E99307242207DFC
:100E2C0020C2AF75430190014C757E10D297C296CB
:100E3C00306204C295C145D294D2AF759F11020E97
:100E4C0099C2AF75430190012A757E40D295C29428
:100E5C00306204C297C165D296D2AF759F10C1990A
:100E6C00207D16C2AF754301900120D297306202EB
:100E7C00C295D2AF759F11C199C2AF754301900154
:100E8C000CD295306202C297D2AF759F10C2662207
:100E9C0090010A757E00D297D295D293C296C294D5
:100EAC00C292C26222788076FF0876FF0876FF082D
:100EBC0076FF08760308760408760B087601087628
:100ECC0001087601788C76010876FF0876FF0876A3
:100EDC00FF0876FF0876FF0876030876FF0876FF92
:100EEC000876FF0876250876D00876FA0876FA0890
:100EFC0076040876FF08760108760008767A08767C
:100F0C00FF087601087601087600087603227887B8
:100F1C00E6FFC2727888E6C394036008C27DE630AF
:100F2C00E102D27DC27E7889E630E102D27EC3EF47
:100F3C0094026008758E01D273020F4D758E00C23B
:100F4C0073227880E6149000809378A4F67881E67A
:100F5C00149000809378A5F67886E61490008D9313
:100F6C0078A6F6789CE67538FF75390CB4020675D0
:100F7C0038A075390AB4030675388275390578A31B
:100F8C00E61490009A93F569D19C22227896E6FAA1
:100F9C007897E6FB7888E6B40305C3EB940EFB3038
:100FAC007F047A007BFFC3EB9AFCC3948250027CD3
:100FBC00827575000575EC8575F0A4C3E5F0947D1C
:100FCC0040F222D27FF1981205917A007B007C10BE
:100FDC00120587E55F2AFA74003BFBDCF37C04C343
:100FEC00EB13FBEA13FADCF7FEC27FF19822E5EF74
:100FFC0020E6037520000520903FFFE520146006D5
:10100C00901DFF1460009304600375EF1253D9BF59
:10101C007581C043FF8012058275EF0243B203E570
:10102C00B3240420E70DF521E5E320E0068521B388
:10103C0043E301120E9C7580FF75A40075F1B27527
:10104C00D4DF7590A975A5FC75F2FE75D50175A652
:10105C000175E241E4F8F6D8FD756B01120EB11280
:0E106C00153878988676753001C2AF12059B54
:10107A001205AB1205911205B21205911205B912A9
:10108A00059112165112059B12059B120596C2AFC5
:10109A0078FA79FA308507D9FBD8F7021C00120FC3
:1010AA001A120F4E120F97120F9878988676120E10
:1010BA009C75885075891275C82475910475D84035
:1010CA0075A82275B80275E690759B80759D0075A6
:1010DA00D10E75BC5875BB0875BA1175E880120532
:1010EA0082D2AF12083B53DACF207E0343DA203094
:1010FA007E0343DA1043DA01C2D8C27112059BD2C9
:10110A00617B037A0CE55E70077A0CDB03021098A8
:10111A00120591207003021098C270E55FC3940211
:10112A0040E1E52F541F856160F561B560D5DAD5D8
:10113A00C26153DACF207E0343DA20307E0343DADA
:10114A0010C2D8C27178A2E67008D274E52F54E0B2
:10115A00F52FC275752900120596307409C3E52961
:10116A00940A4002D2751205877802307402780018
:10117A00C3E55F9840F0C2AF1205AB1205AB12058A
:10118A00ABD2AF12059B754D007888E6B4030241D5
:10119A0078120587788CE6C394015003021278E529
:1011AA0030C394015003021278207435C3E55F946A
:1011BA00FF5003021278C2AF1205C0D2AF120596D1
:1011CA00C3E55F940150EFC2AF1205AB12058C1252
:1011DA0005ABD2AF120596C3E55F94FF40E902164C
:1011EA00D67F05D27F120F98120596C2AFC27F1220
:1011FA000F98AE5FC3E55F947FD2AF407B12058242
:10120A00C2AF1205C0D2AFDFDA120FCFC3EE940518
:10121A007897F612059B12157A1216597F0AD27F11
:10122A00120F98120596C2AFC27F120F98AE5FC313
:10123A00E55F947FD2AF50E4120582C2AF1205ABCC
:10124A0012058C1205ABD2AFDFD4120FCFEE2405F4
:10125A007896F612059B12157A12168812059612BE
:10126A000F98C3E55F94FF500221B30216D6C3E577
:10127A005F954D4003855F4D12059678017988E7A1
:10128A00B403027805C3E55F9840022193C2AF1206
:10129A0005C01205C01205C0D2AF12059B753000F9
:1012AA00E4F531F5320531E531F470390532789AD1
:1012BA00E67819146012783214600D787D1460088B
:1012CA0078FA146003753200C3E532984017153274
:1012DA007531B478998676C2AF1205C0D2AF7898C4
:1012EA00867612059612058CE52A7005307402017D
:1012FA009878012074027806C3E55F9840A7788839
:10130A00E6C394036003120596E52A700302109857
:10131A00C2AF120E9CE4F522F523F524F525F52635
:10132A00F56AD2AF7885E6C333F568E4F545F54644
:10133A00F547F548F549F573F52CF52DF53775732D
:10134A000875BB1012058212083FE5E820ECFBA8DD
:10135A00BDA9BEE97001F88874120843757308754F
:10136A00BB107887E6FE7602120F1A7887EEF6C26D
:10137A00AF7564FF1208BB852264852265852266E3
:10138A00D2AF752201752401752501752601856381
:10139A006C756D017888E6B40307C27D307602D297
:1013AA007DD268D269753300120E02120E27120816
:1013BA00DB1208E21208DB1208E21208DB0213D77A
:1013CA00C2AF120F1AD2AF75730075BB08120B6643
:1013DA0012068B120C80120CCA1208E2120B55303C
:1013EA006D0312068C2067031207DE3067031208AA
:1013FA0025120C80120CEF1208E2120B66306D03F4
:10140A001206C8120C80120D661208E2120B553031
:10141A006D03120726120C80120D8B1208E2120BB2
:10142A0066306D03120783120C80120E021208E254
:10143A0012083F120B55120C80120E271208431283
:10144A0008E2306932206B2F85676485676585639A
:10145A006C756D0179187A0CC3E53399400CC26931
:0F146A00D26A8A357564FF021481C3E55F94016D
:1014790040030213D70214FE306A1B206B18E535AE
:10148900147004C26A61CAF535C3E55F940140036B
:101499000213D70214FE753600C3E56278829850AC
:1014A90054307404E52A604D7888E6B40317207D2A
:1014B9000520760781CE30760281CE206B07D26B6C
:1014C900856764811678F0306B058567647820C379
:1014D900E54198500261D7306B1BC26BC27D3076F3
:1014E90002D27DD26A75351285676461D70536E502
:1014F9005F6002A101753600C2AF120E9C7887E6C3
:10150900FE7602120F1A7887EEF6E4F522F523F536
:1015190024F525F526F568C268D2AF120582120EA8
:101529009C307409C3E53694054002019841AA909C
:101539001A0D78201215BCE520B45A0CA31215BC5B
:10154900E520B4A50302155A120EB112157A021537
:1015590079901A0378807B0A1215BCA308DBF990ED
:101569001A0F788C7B181215BCA308DBF9901A277F
:1015790022C2AF1215FB1215D5901A00740E12155E
:10158900C1A374041215C1A374141215C1901A03CE
:1015990078807B0A1215C0A308DBF9901A0F788CA2
:1015A9007B181215C0A308DBF912160E1215EC9060
:1015B9001A2722E493F622E6438F01538FFD75EF34
:1015C9000275B7A575B7F1F0538FFE22438F024319
:1015D9008F0175EF0275B7A575B7F1901A0DF05324
:1015E9008FFC22901A0D745AB1C1901A0E74A5B1CC
:1015F900C1227A3079D07820901A40B1BCE520F721
:1016090009A3DAF7227A3079D0901A40E7B1C109F3
:10161900A3DAF922AB77A878BB01027984BB02026D
:101629007985BB03027986BB04027992BB050279ED
:1016390087BB060279A3BB0702799CBB080279889C
:10164900BB09027989E8F7227C0512059BDCFB229C
:10165900C2AF1205AB1205B21205B91205C01205C7
:101669008C1205AB1205B21205B91205C012058C10
:101679001205AB1205B21205B91205C0D2AF22C2CA
:10168900AF1205C01205B91205B21205AB12058CCD
:101699001205C01205B91205B21205AB12058C125A
:1016A90005C01205B91205B21205ABD2AF22AE7749
:1016B900AF78C2AF1205AB1205AB1205AB12058CA0
:1016C900DEF21205C012058CDFF8D2AF22D159D152
:1016D90051D151757701757801757900D1B77C05BC
:1016E900AD5F12059BC3ED955F70F5C3E55F94018E
:1016F900400AC3E55F94FF4032021712D11DB17A47
:10170900D159C2AF75EF12D151DCD50579C3E5794D
:101719009403500280C6D1510578E5771490009F53
:1017290093F808C3E57898500280AED151D151059C
:1017390077C3E577940A5002809C120EB1B17AC240
:06174900AF75EF12D15153
:0319FD00020FFADC
:101A00000E0414FFFFFFFF03040B0101015AA5019F
:101A1000FFFFFFFFFF03FFFFFF25D0FAFA04FF01DE
:081A2000007AFF01010003FF41
:101A4000235475726E69677931304123202020203C
:101A500023424C48454C4923463333302320202031
:101A60002020202020202020202020202020202076
:101C0000C2AFC2D353D9BF7581C043B20343FF8073
:101C1000752438752503B1C975EF0275E24043F1AB
:101C20002053A4DF75D400D2857DFA780379E67C51
:101C300010752200752300901DD67B0675249875BB
:101C400025013085028142208508D8FBD9F9DCF7CF
:101C500081B4308508D8FBD9F9DCF781B4B189E4C7
:101C600093A3C39A6004DDC381B4DBDBB17B600264
:101C7000812B7B08E493FAA3B15CDBF87A30B15C8A
:101C8000752200752300B17BEAFCEBFDC3ED94FEE9
:101C9000400EB17B8A278B28ED30E0048A828B834B
:101CA000B17B7AC270D8C3ED94FE601350CEBD00F4
:101CB00025EC60097520007521FF0200008100A855
:101CC00027A9280809D804D90281D3B17FEA89AAB3
:101CD000F281C50D81A0C3ED94035049EDA2E092BD
:101CE000007AC5C3E5829400E583941C50902000DF
:101CF00010438F02438F0175B7A575B7F1F030001F
:101D00001FA827A9280809438F01538FFDD804D99C
:101D100002A12089AAE275B7A575B7F1F0A3A10DBC
:101D2000538FFC817C7AC1BD030CE493A3FAB140CC
:101D3000DCF8B138817C817EAA22AB23B15CEBFA5E
:101D4000EA6222752608C3E52313F523E52213F57D
:101D50002250066323A0632201D526EAB1C9B1C986
:101D600075260AEAF4200102D285300102C285B14B
:101D7000C9C3134002C201D526EB22B17FEAFB2082
:101D80008502A17F308502A184752608AE24AF2587
:101D9000C3EF13FFEE13FEB1CDB1C9C3EA13308513
:101DA000024480FA30E703632201C3E52313F523DD
:101DB000E52213F52250066323A0632201D526D91C
:101DC000E52265236523F52222AE24AF250E0FDE22
:101DD000FEDFFCD20122424C48656C693437316326
:041DE000F3300601D5
:00000001FF
